:1000000003C003C003C003C003C003C003C003C0D8
:1000800042C464C463C462C461C460C45FC45EC467
:100090005DC45CC45BC45AC459C458C457C422C0AC
:1000A00040C06CC03EC03DC03CC03BC03AC039C03F
:1000B00038C037C036C035C034C033C0040309046B
:1000C00012011001FF000008D016530706010000BE
:1000D0000001090212000101008032090400000041
:1000E0000000000011241FBECFE5D2E0DEBFCDBF6F
:1000F00000EB0F9307E00F9310E0A0E6B0E0E2EE14
:10010000FFE102C005900D92A636B107D9F710E0C5
:10011000A6E6B0E001C01D92AC39B107E1F7E7D126
:10012000EDC3BDCFA82FB92F80E090E041E050EAA9
:10013000609530E009C02D9182279795879510F042
:1001400084279527305EC8F36F5FA8F30895EADF30
:100150008D939D930895A6E088279927AA9569F025
:100160000197E1F3B399FCCFB39BFECF81E09927D0
:10017000A6B3019611F0A871D9F70895CF93CFB720
:10018000CF93C0915F02C03B21F4C0915E02C730A3
:1001900021F0CF91CFBFCF9181CFCC27C395B39B17
:1001A000E9F7B39B0BC0B39B09C0B39B07C0B39BDC
:1001B00005C0B39B03C0B39B01C0D3C00F92DF93B4
:1001C000C0917F00DD27CA57DF4F012EB39B03C0CC
:1001D000DF910F90E6CF2F930F931F934F932FEF45
:1001E0004F6F06B303FB20F95F933F9350E03BE072
:1001F00065C016B30126502953FDC89556B3012793
:1002000003FB25F92F7306B3B1F05027102713FB1A
:1002100026F906B22230F0F000C016B3012703FB26
:1002200027F90126502906B22430E8F54F772068D7
:1002300016B30000F6CF50274F7D206206B2102F74
:10024000000000C006B300265029102713FB26F932
:1002500006B2E2CF4F7B06B3206400C0DACF01269E
:100260005029187106B269F14E7F2160012F16B333
:1002700028C0002650294D7F06B22260102F29C0C9
:10028000012650294B7F06B22460012F2DC016B3E2
:1002900001265029477F2860000006B22EC04F7EFD
:1002A00006B3206130C0422706B349930026502987
:1002B000102706B24FEF13FB20F9297F16B379F20E
:1002C000187159F10126502906B2012703FB21F9C3
:1002D000237F06B371F2002650293150D0F006B2C8
:1002E000102713FB22F9277E16B351F2012650295D
:1002F000012703FB06B223F92F7C49F2000006B365
:10030000102713FB24F90026502906B22F7939F261
:1003100070CF10E21ABF002717C03B503195C31BA6
:10032000D04010E21ABF0881033CF9F00B34E9F029
:1003300020917D001981110F1213EDCF093651F173
:100340000D3211F0013E39F7009384003F915F9127
:100350004F911F910F912F91DF910F90CAB7C5FD5B
:100360001DCFCF91CFBFCF9118952091840022232C
:1003700069F310918200112321F5343022F130937A
:10038000820020937E0010917F003BE0311B309370
:100390007F0019C00091820001309CF40AE5309181
:1003A000600034FD11C000936000C2E7D0E010C0CF
:1003B000052710E000C021C0052710E0C89508BB44
:1003C00014C03AE501C032ED032EC0E0D0E032E0C7
:1003D00017B31861C39A08B317BB58E120E84FEF71
:1003E00020FF052708BB279517951C3F28F700001D
:1003F0004552B0F720FF0527279508BB17951C3FEE
:10040000B8F629913A9561F7077E10918300110F94
:1004100008BBC250D04011F010937D0010E21ABF0B
:10042000086017B3177E402F477E54E05A95F1F7C6
:1004300008BB17BB48BB8ACF81E080936900F89462
:10044000E0917000F0917100329785E08093570041
:10045000E89507B600FCFDCF789408959C01E091E3
:100460007000F0917100309789F1E430F105F1F0FE
:1004700087E1EC37F80739F420916C0030916D007A
:100480002E5B3B4F15C087E1EE37F80739F420911A
:100490006E0030916F002D5B3B4F0AC087E1EA3759
:1004A000F80731F481B7282F30E002C02FEB3BEC86
:1004B000F89481E0090180935700E895112478941D
:1004C0003296F0937100E0937000089581E180937B
:1004D0005700E895EBCF8FEF9FEFC0DF8091700062
:1004E000909171008F739070892BA9F7A5CF1F93FE
:1004F000CF93DF9388E10FB6F89481BD11BC0FBE96
:10050000E0E0F0E0859194918F5B9B4C39F4E4E05E
:10051000F0E0859194918F5B9B4C09F0DCDF1092A9
:10052000710010927000BD9AC59A82E291EA01971B
:10053000F1F7B5997DC1AC9A8BB780628BBFBB9A3E
:1005400088E893E1ECE9F1E03197F1F70197D1F711
:10055000BB98789410918200135017FDD4C08091FD
:100560007F00CCE0D0E0C81BD109CA57DF4F809193
:100570007E008D3209F091C0183009F0C2C083ECC2
:10058000809372008AE58093600010926B0028814E
:10059000822F80769981882329F11092670010922A
:1005A0006600992341F482E690E090938100809365
:1005B000800024E068C0913051F48C819D8190933B
:1005C00071008093700027FD59C09FEF58C0809143
:1005D0006800923011F4816001C0846080936800EB
:1005E00020E051C08A8110927B00992331F410924F
:1005F0007C008BE790E022E03CC0953019F48093BA
:10060000830034C0963011F58B81813019F482EA71
:1006100097E104C0823041F484EB97E1909381002C
:100620008093800022E10EC0833059F48A818823B0
:1006300041F48EE997E1909381008093800024E05B
:1006400001C020E080E480936B001DC0983019F455
:1006500085E890E009C0993019F48093850006C0C0
:100660009A3021F48BE790E021E003C08BE790E023
:1006700020E0909381008093800005C09E8180E8F7
:1006800080936B0007C08F81882319F49E81921795
:1006900008F0922F9093610034C080916B0087FF27
:1006A00030C08091700090917100009739F488817A
:1006B000998190936D0080936C000DC084309105FA
:1006C00039F48881998190936F0080936E0003C004
:1006D0008058974138F488819981C0DE125011F01A
:1006E0002296DFCF80917000909171008F7390708F
:1006F000892B39F4809168008260809368001092A1
:100700006100109282008091600084FF3CC0809163
:1007100061008F3FC1F1182F893008F018E0811B6C
:10072000809361008091720098E88927809372001D
:100730001123E1F0E0918000F091810080916B0045
:1007400086FF09C0912FA3E7B0E084918D93319685
:100750009150D9F707C0912FA3E7B0E081918D9315
:100760009150E1F7F0938100E093800083E790E0FF
:10077000612FEDDC612F6C5F6C3019F08FEF80938F
:1007800061006093600094E186B3887131F4915008
:10079000D9F71092830010927D0010E0992309F49C
:1007A00011E080916A00811739F0112319F4F8944F
:1007B00066D0789410936A008CE991E00197F1F784
:1007C00080916600909167000196909367008093F6
:1007D000660080916800182F80FF14C0F894E0E84C
:1007E000F7E1E054F04083E080935700E89507B6C6
:1007F00000FCFDCF3097A9F71092710010927000A5
:100800006ADE789411FF0FC08AE390E20197F1F756
:1008100080917000909171008F739070892B11F00E
:100820005ADE01C009DE12FD03C01092680092CEAC
:1008300082E291EA0197F1F718BA17BAF8941BBE51
:1008400015BA10925F0210925E02EAE7F7E1949106
:10085000892F81508E3F20F00DC081B7815081BF1C
:1008600081B79817D0F303C081B78F5F81BF81B77D
:100870008917D0F312CCDF91CF911F910895FF9289
:100880000F931F93CF93DF9380E8F82E00E0C0E032
:10089000D0E0102F1F0D11BF5EDC29E084339207DA
:1008A0000CF0102FF6942196C830D10511F0012FCD
:1008B000F0CF115011BF1F5F012FEC0110C04BDCB6
:1008C0008453994097FF03C0909581959F4F8C1753
:1008D0009D0714F401B7EC0181B78F5F81BF21B789
:1008E00030E0812F90E001968217930744F701BF13
:1008F000DF91CF911F910F91FF900895F894FFCF52
:100900005AFF177C400800000000000000000000B3
:1009100000000000000000000000000000000000D7
:1009200000000000000011241FBECFE5D2E0DEBFB2
:10093000CDBF10E0A0E6B0E0EEECFBE002C0059019
:100940000D92A236B107D9F720D13FC199CB05C08E
:10095000EDE1F0E13197F1F701970097C9F70895BC
:10096000AC01407C20E030E0F901E40FF51F8591F7
:100970009491F901EE7FE60FF71F918380832E5F3C
:100980003F4F2034310581F70895FC01E07C83E07E
:1009900080935700E89507B600FCFDCF0895CF93EC
:1009A000DF93EC01A0E0B0E0AD014C0F5D1FFB0157
:1009B000EA0FFB1F8081918121E0FA010C01209355
:1009C0005700E89511241296A034B10569F785E027
:1009D000FE0180935700E89507B600FCFDCFDF913C
:1009E000CF910895DF93CF93CDB7DEB7C054D040F9
:1009F0000FB6F894DEBF0FBECDBF209160003091DE
:100A000061003695279521503044FE01319621939F
:100A10003193CE018F5B9F4FE817F907C1F780E054
:100A200090E0B3DF80E090E0BE016F5F7F4FB7DF03
:100A3000C05CDF4F0FB6F894DEBF0FBECDBFCF91C5
:100A4000DF910895EF92FF920F931F93DF93CF935F
:100A5000CDB7DEB7C054D0400FB6F894DEBF0FBE9E
:100A6000CDBF00E010E035C09B01359527957E0194
:100A70000894E11CF11C89E0A630B80738F0220F79
:100A8000331FE20EF31E8FEF9FEF07C0FD0185912C
:100A90009491220F331FE20EF31EF701918380839E
:100AA0006E5F7F4F129660347105F1F680916000A1
:100AB00090916100800F911F68DF8091600090919C
:100AC0006100800F911FBE016F5F7F4F68DF005C88
:100AD0001F4FF8E000381F0731F0D801A256BF4F72
:100AE00060E070E0C1CFC05CDF4F0FB6F894DEBFAE
:100AF0000FBECDBFCF91DF911F910F91FF90EF906F
:100B00000895DF93CF93CDB7DEB7C054D0400FB672
:100B1000F894DEBF0FBECDBF80E090E0BE016F5FF6
:100B20007F4F1EDF80E090E0019680329105E1F773
:100B30008FEF9FEF9A83898380E090E026DF80E04B
:100B400090E0BE016F5F7F4F2ADFC05CDF4F0FB6C2
:100B5000F894DEBF0FBECDBFCF91DF91089587B36C
:100B6000836087BBC19820E08DE190E1FC01319763
:100B7000F1F7C19A0197F1F7C1982F5F2A3FA1F7CA
:100B80000895E0E0F0E00995089588B318BA87B3B6
:100B90008FEF87BB8AEF90E0EDE1F0E13197F1F75D
:100BA0000197D1F787B317BA8AEF90E0EDE1F0E152
:100BB0003197F1F70197D1F7F894A3DF43DF12DF04
:0E0BC000CEDFDFDF80E090E00895F894FFCFF5
:020BCE0080178E
:040000030000008079
:00000001FF
